:020000040800F2
:1000000000060020E1020008E3020008E302000805
:10001000E3020008E3020008E3020008E30200082C
:10002000E3020008E3020008E3020008F1200008F0
:10003000E3020008E3020008E3020008E30200080C
:10004000E3020008E3020008E3020008E3020008FC
:10005000E3020008E3020008BD240008E9240008C8
:1000600015250008412500086D250008E302000859
:10007000E3020008E3020008E3020008E3020008CC
:10008000E3020008E3020008E3020008E3020008BC
:10009000E3020008E3020008E302000899250008D3
:1000A000E3020008E3020008E3020008E30200089C
:1000B000E3020008E3020008E3020008E30200088C
:1000C000E3020008E3020008E3020008E30200087C
:1000D000E3020008E3020008E3020008E30200086C
:1000E000FD250008E3020008E3020008E30200081F
:1000F000E3020008E3020008E3020008E30200084C
:10010000E3020008E302000899260008E302000861
:10011000E3020008E3020008E3020008E30200082B
:10012000E3020008E3020008E3020008E30200081B
:10013000E3020008E3020008E3020008E30200080B
:10014000E3020008E3020008E3020008E3020008FB
:10015000E3020008E3020008E3020008E3020008EB
:10016000E3020008E3020008E3020008E3020008DB
:10017000E3020008E3020008E3020008E3020008CB
:10018000E3020008E3020008712600088526000843
:10019000E3020008E3020008E3020008E3020008AB
:1001A000E3020008E3020008E3020008E30200089B
:1001B000E3020008E3020008E3020008E30200088B
:1001C000E3020008E3020008E3020008E30200087B
:1001D000E3020008E3020008E3020008E30200086B
:1001E000E3020008E3020008E3020008E30200085B
:1001F000E3020008E3020008E3020008E30200084B
:10020000E3020008E3020008E3020008E30200083A
:10021000E3020008E3020008E3020008E30200082A
:10022000E3020008E3020008E3020008E30200081A
:10023000E3020008E3020008E3020008E30200080A
:10024000E3020008E3020008E3020008E3020008FA
:10025000E3020008E3020008E3020008E3020008EA
:10026000E3020008E3020008E3020008E3020008DA
:10027000E3020008E3020008E3020008E3020008CA
:10028000E3020008E3020008E3020008E3020008BA
:10029000E3020008E3020008E3020008E3020008AA
:1002A000E3020008E3020008E3020008E30200089A
:1002B000E3020008E3020008E3020008E30200088A
:1002C000E3020008E3020008E3020008E30200087A
:1002D000E3020008E3020008E3020008E30200086A
:1002E00002E000F000F8FEE772B6374880F30888B5
:1002F000364880F3098836483649086040F20000E5
:10030000CCF200004EF63471CEF200010860BFF36B
:100310004F8FBFF36F8F40F20000C0F2F0004EF637
:100320008851CEF200010860BFF34F8FBFF36F8F8B
:100330004FF00000E1EE100A4EF63C71CEF20001E3
:100340000860062080F31488BFF36F8F01F028FD4A
:1003500001F02AFE4FF055301F491B4A91423CBF25
:1003600041F8040BFAE71D49184A91423CBF41F895
:10037000040BFAE71A491B4A1B4B9A423EBF51F83D
:10038000040B42F8040BF8E700201849184A914280
:100390003CBF41F8040BFAE701F040FD01F086FE96
:1003A000144C154DAC4203DA54F8041B8847F9E7A6
:1003B00000F042F8114C124DAC4203DA54F8041B21
:1003C0008847F9E701F028BD000600200022002040
:1003D0000000000808ED00E00000002000060020FA
:1003E000582900080022002030220020302200205E
:1003F000702F0020E0020008E0020008E002000880
:10040000E00200082DE9F04F2DED108AC1F80CD064
:10041000D0F80CD0BDEC108ABDE8F08F002383F338
:1004200011882846A047002001F08CF9FEE701F072
:10043000FFF800DFFEE7000038B500F0ADFB01F08B
:100440006FFC054601F0A2FC0446D0B90F4B9D425B
:1004500019D001339D4242F2107512BF04460025A7
:100460000124002001F066FC0CB100F077F800F0E8
:1004700023FD00F0EFFB284600F0F0F800F06EF8E6
:10048000F9E70025EDE70546EBE700BF010007B0FF
:1004900008B500F0ABFBA0F120035842584108BD5D
:1004A00007B541F21203022101A8ADF8043000F0B3
:1004B000BBFB03B05DF804FB38B5302383F3118830
:1004C000174803680BB101F0FBF90023154A4FF4FC
:1004D0007A71134801F0EAF9002383F31188124C72
:1004E000236813B12368013B2360636813B1636819
:1004F000013B63600D4D2B7833B963687BB90220F3
:1005000000F070FC322363602B78032B07D1636803
:100510002BB9022000F066FC4FF47A73636038BD9B
:1005200030220020B9040008502300204822002077
:10053000084B187003280CD8DFE800F00805020803
:10054000022000F045BC022000F038BC024B002223
:100550005A6070474822002050230020F8B5394BDC
:10056000394A1C46196801316BD004339342F9D1E2
:100570006268364B9A4264D9354B9B6803F100633D
:1005800003F500339A425CD2002000F089FB022080
:10059000FFF7CEFF2F4B00219A6C99641A6F1967F1
:1005A0001A6FDA6CD9645A6F59675A6F1A6D1965E8
:1005B0009A6F99679B6F72B64FF0E023C3F8084DAE
:1005C000D4E90004BFF34F8FBFF36F8F224AC2F804
:1005D0008410BFF34F8F536923F480335361BFF30B
:1005E0004F8FD2F8803043F6E076C3F3C905C3F3EA
:1005F0004E335B0103EA060C29464CEA8177013948
:10060000C2F87472F9D2203B13F1200FF2D1BFF37C
:100610004F8FBFF36F8FBFF34F8FBFF36F8F536950
:1006200023F4003353610023C2F85032BFF34F8FDD
:10063000BFF36F8F302383F31188854680F30888DA
:100640002047F8BD0000020820000208FFFF010853
:10065000002200200045025800ED00E02DE9F04F97
:1006600093B0B44B2022FF2100900AA89D6800F0AF
:10067000CDFBB14A1378A3B90121B04811700360D2
:10068000302383F3118803680BB101F019F90023BB
:10069000AB4A4FF47A71A94801F008F9002383F3BB
:1006A0001188009B13B1A74B009A1A60A64A1378D1
:1006B000032B03D000231370A24A53604FF0000AAB
:1006C000009CD3465646D146012000F081FB24B160
:1006D0009C4B1B68002B00F02682002000F086FA5D
:1006E0000390039B002BF2DB012000F067FB039BD0
:1006F000213B1F2BE8D801A252F823F07D07000808
:10070000A507000839080008C9060008C90600083E
:10071000C9060008CB0800089B0A0008B5090008B4
:10072000170A00083F0A0008650A0008C906000801
:10073000770A0008C9060008E90A00081D08000831
:10074000C90600082D0B0008890700081D080008CD
:10075000C9060008170A0008C9060008C9060008EB
:10076000C9060008C9060008C9060008C90600082D
:10077000C9060008C9060008390800080220FFF76A
:1007800087FE002840F0F981009B022105A8BAF1FC
:10079000000F08BF1C4641F21233ADF8143000F0D0
:1007A00043FA91E74FF47A7000F020FA071EEBDB72
:1007B0000220FFF76DFE0028E6D0013F052F00F272
:1007C000DE81DFE807F0030A0D101336052304214C
:1007D00005A8059300F028FA17E004215548F9E729
:1007E00004215A48F6E704215948F3E74FF01C0862
:1007F000404608F1040800F055FA0421059005A8C8
:1008000000F012FAB8F12C0FF2D101204FF00009DC
:1008100000FA07F747EA0B0B5FFA8BFB00F042FB8D
:1008200026B10BF00B030B2B08BF0024FFF738FE9B
:100830004AE704214748CDE7002EA5D00BF00B0373
:100840000B2BA1D10220FFF723FE074600289BD0E7
:100850000120002600F024FA0220FFF769FE5FFA6B
:1008600086F8404600F02CFA0446B0B103994046A1
:100870000136A1F140025142514100F031FA002805
:10088000EDD1BA46044641F21213022105A83E46B4
:10089000ADF8143000F0C8F916E725460120FFF73F
:1008A00047FE244B9B68AB4207D9284600F0FAF973
:1008B000013040F067810435F3E70025224BBA464A
:1008C0003E461D701F4B5D60A8E7002E3FF45CAFF5
:1008D0000BF00B030B2B7FF457AF0220FFF728FE22
:1008E000322000F083F9B0F10008FFF64DAF18F0A8
:1008F00003077FF449AF0F4A08EB05039268934260
:100900003FF642AFB8F5807F3FF73EAF124BB84598
:10091000019323DD4FF47A7000F068F90390039A95
:10092000002AFFF631AF039A0137019B03F8012B30
:10093000EDE700BF002200204C23002030220020E1
:10094000B90400085023002048220020042200207F
:10095000082200200C2200204C220020C820FFF793
:1009600097FD074600283FF40FAF1F2D11D8C5F1A2
:1009700020020AAB25F0030084494245184428BFF1
:100980004246019200F038FA019AFF217F4800F0B8
:100990003DFA4FEAA803C8F387027C492846019331
:1009A00000F03CFA064600283FF46DAF019B05EBD2
:1009B000830533E70220FFF76BFD00283FF4E4AE28
:1009C00000F0ACF900283FF4DFAE0027B846704BCA
:1009D0009B68BB4218D91F2F11D80A9B01330ED038
:1009E00027F0030312AA134453F8203C0593404612
:1009F000042205A9043700F087FA8046E7E7384665
:100A000000F050F90590F2E7CDF81480042105A814
:100A100000F00AF902E70023642104A8049300F01F
:100A2000F9F800287FF4B0AE0220FFF731FD00286E
:100A30003FF4AAAE049800F067F90590E6E70023BA
:100A4000642104A8049300F0E5F800287FF49CAE2C
:100A50000220FFF71DFD00283FF496AE049800F039
:100A600055F9EAE70220FFF713FD00283FF48CAEAA
:100A700000F064F9E1E70220FFF70AFD00283FF4E7
:100A800083AE05A9142000F05FF907460421049005
:100A900004A800F0C9F83946B9E7322000F0A6F8FA
:100AA000071EFFF671AEBB077FF46EAE384A07EB48
:100AB0000903926893423FF667AE0220FFF7E8FC15
:100AC00000283FF461AE27F003074F44B9453FF4D7
:100AD000A5AE484609F1040900F0E4F804210590A8
:100AE00005A800F0A1F8F1E74FF47A70FFF7D0FC09
:100AF00000283FF449AE00F011F9002844D00A9BC9
:100B000001330BD008220AA9002000F087F9002841
:100B10003AD02022FF210AA800F078F9FFF7C0FCA4
:100B20001C4800F015FE13B0BDE8F08F002E3FF416
:100B30002BAE0BF00B030B2B7FF426AE00236421AE
:100B400005A8059300F066F8074600287FF41CAE60
:100B50000220FFF79DFC804600283FF415AEFFF70A
:100B60009FFC41F2883000F0F3FD059800F0B2F9E7
:100B700046463C4600F096F9A6E506464EE64FF09E
:100B8000000901E6BA467EE637467CE64C220020A4
:100B900000220020A086010070470000104B70B5B5
:100BA0001B780C460133DBB2012B12D80D4B1D68AC
:100BB0004FF47A732968A2FB033222460E6A01467B
:100BC0002846B047844204D1074B002201201A7006
:100BD00070BD4FF4FA7000F0BBFD0020F8E700BFD5
:100BE00010220020142200209C230020002307B59F
:100BF000024601210DF107008DF80730FFF7CEFF07
:100C000020B19DF8070003B05DF804FB4FF0FF3002
:100C1000F9E700000A46042108B5FFF7BFFF80F09E
:100C20000100C0B2404208BD074B0A4630B41978F3
:100C3000064B53F82140014623682046DD69044BEA
:100C4000AC4630BC604700BF9C230020142200202B
:100C5000A086010070B5104C0025104E00F038FF42
:100C600020803068238883420CD8002520880138F2
:100C700000F02AFF23880544013BB5F5802F23802F
:100C8000F4D370BD00F020FF336805440133B5F59F
:100C9000003F3360E5D3E8E79E230020582300207F
:100CA00000F0F4BF00F1006000F50030006870470C
:100CB00000F10060920000F5003000F06BBF000012
:100CC000054B1A68054B1B889B1A834202D91044B6
:100CD00000F0FABE00207047582300209E23002019
:100CE00038B50446074D29B128682044BDE838408E
:100CF00000F002BF2868204400F0ECFE0028F3D08A
:100D000038BD00BF582300200020704700F1FF507D
:100D100000F58F10D0F8000870470000064991F8E0
:100D2000243033B100230822086A81F82430FFF709
:100D3000BFBF0120704700BF5C230020014B186833
:100D4000704700BF0010005C194B013803220844B3
:100D500070B51D68174BC5F30B042D0C1E88A642F9
:100D60000BD15C680A46013C824213460FD214F94B
:100D7000016F4EB102F8016BF6E7013A03F1080387
:100D8000ECD181420B4602D22C2203F8012B042421
:100D9000094A1688AE4204D1984284BF967803F877
:100DA000016B013C02F10402F3D1581A70BD00BF7F
:100DB0000010005C18220020B8270008022803D188
:100DC000024B4FF080629A61704700BF000C0258DE
:100DD000022803D1024B4FF480629A61704700BF32
:100DE000000C0258022804D1024A536983F480633C
:100DF00053617047000C0258002310B5934203D092
:100E0000CC5CC4540133F9E710BD00000244034632
:100E1000934202D003F8011BFAE770472DE9F8432B
:100E20001F4D14460746884695F8242052BBDFF82C
:100E300070909CB395F824302BB92022FF214846AE
:100E40002F62FFF7E3FF95F824004146C0F1080246
:100E500005EB8000A24228BF2246D6B29200FFF7DF
:100E6000CBFF95F82430A41B17441E449044E4B2F1
:100E7000F6B2082E85F82460DBD1FFF74FFF00287B
:100E8000D7D108E02B6A03EB82038342CFD0FFF770
:100E900045FF0028CBD10020BDE8F8830120FBE707
:100EA0005C230020024B1A78024B1A70704700BF77
:100EB0009C23002010220020034B04490B60044BAC
:100EC000186800F01BBB00BF80841E008423002034
:100ED00014220020094B1822002110B504461846A0
:100EE000FFF794FF064A074B01461278046053F857
:100EF0002200BDE8104000F001BB00BF84230020A9
:100F00009C2300201422002030B50A44084D914251
:100F10000DD011F8013B5840082340F30004013B79
:100F20002C4013F0FF0384EA5000F6D1EFE730BD08
:100F30002083B8ED026843681143016003B118478C
:100F400070470000024A136843F0C0031360704703
:100F500000780040024A136843F0C00313607047F2
:100F6000007C004037B51A4C1A4D204600F0BAFA02
:100F700004F11400009400234FF40072164900F0AD
:100F800077F94FF40072154904F138000094144BBE
:100F900000F0F0F9134BC4E91735134C204600F06C
:100FA000A1FA04F1140000234FF400720F490094D9
:100FB00000F05EF90E4B4FF400720E4904F1380058
:100FC000009400F0D7F90C4BC4E9173503B030BDDD
:100FD000A023002000E1F5057824002078280020D7
:100FE000450F0008007800400C24002078260020DF
:100FF000550F0008782A0020007C0040037C30B5A3
:10100000274C002918BF0C46012B0CD1254B9842C8
:1010100036D1254B9A6C42F080429A641A6F42F0A6
:1010200080421A671B6F2268036EC16D03EB520387
:101030008466B3FBF2F36268150442BF23F0070530
:1010400003F0070343EA4503CB60A36843F0400382
:101050004B60E36843F001038B6042F4967343F006
:1010600001030B604FF0FF330B62510505D512F001
:10107000102211D0B2F1805F10D080F8643030BD02
:101080000A4B9842CFD1084B9A6C42F000429A64C6
:101090001A6F42F00042C4E77F23EEE73F23ECE7FC
:1010A000C8270008A0230020004502580C24002077
:1010B0002DE9F047C66D05463768F46921073462AB
:1010C0001AD014F0080118BF4FF48071E20748BF2E
:1010D00041F02001A3074FF0300348BF41F0400129
:1010E000600748BF41F0800183F31188281DFFF796
:1010F00021FF002383F31188E2050AD5302383F30F
:1011000011884FF48061281DFFF714FF002383F33B
:1011100011884FF030094FF0000A14F0200838D140
:101120003B0616D54FF0300905F1380A200610D5D8
:1011300089F31188504600F051F9002836DA082169
:10114000281DFFF7F7FE27F080033360002383F3A9
:101150001188790614D5620612D5302383F31188DD
:10116000D5E913239A4208D12B6C33B127F04007FD
:101170001021281DFFF7DEFE3760002383F311885E
:10118000E30618D5AA6E1369ABB15069BDE8F04704
:10119000184789F31188736A284695F86410194036
:1011A00000F0BAF98AF31188F469B6E7B06288F3FF
:1011B0001188F469BAE7BDE8F0870000F8B5154674
:1011C000826804460B46AA4200D28568A169266956
:1011D000761AB5420BD218462A46FFF70DFEA369D0
:1011E0002B44A3612846A3685B1BA360F8BD0CD900
:1011F000AF1B18463246FFF7FFFD3A46E168304420
:10120000FFF7FAFDE3683B44EBE718462A46FFF791
:10121000F3FDE368E5E7000083689342F7B5044611
:10122000154600D28568D4E90460361AB5420BD25F
:101230002A46FFF7E1FD63692B4463612846A368F2
:101240005B1BA36003B0F0BD0DD93246AF1B01910B
:10125000FFF7D2FD01993A46E0683144FFF7CCFD33
:10126000E3683B44E9E72A46FFF7C6FDE368E4E7A5
:1012700010B50A440024C361029B8460C16002610E
:101280000362C0E90000C0E9051110BD08B5D0E94E
:101290000532934201D1826882B98268013282604C
:1012A0005A1C426119700021D0E904329A4224BFCD
:1012B000C368436100F068FA002008BD4FF0FF30BA
:1012C000FBE7000070B5302304460E4683F3118817
:1012D000A568A5B1A368A269013BA360531CA361E3
:1012E00015782269934224BFE368A361E3690BB1D7
:1012F00020469847002383F31188284607E03146AB
:10130000204600F031FA0028E2DA85F3118870BD3A
:101310002DE9F74F04460E4617469846D0F81C9024
:101320004FF0300A8AF311884FF0000B154665B173
:101330002A4631462046FFF741FF034660B9414641
:10134000204600F011FA0028F1D0002383F3118821
:10135000781B03B0BDE8F08FB9F1000F03D0019006
:101360002046C847019B8BF31188ED1A1E448AF36F
:101370001188DCE7C160C361009B82600362C0E941
:1013800005111144C0E9000001617047F8B5044639
:101390000D461646302383F31188A768A7B1A368CA
:1013A000013BA36063695A1C62611D70D4E9043279
:1013B0009A4224BFE3686361E3690BB12046984712
:1013C000002080F3118807E03146204600F0CCF978
:1013D0000028E2DA87F31188F8BD0000D0E9052380
:1013E00010B59A4201D182687AB98268002101322F
:1013F00082605A1C82611C7803699A4224BFC368C8
:10140000836100F0C1F9204610BD4FF0FF30FBE7CB
:101410002DE9F74F04460E4617469846D0F81C9023
:101420004FF0300A8AF311884FF0000B154665B172
:101430002A4631462046FFF7EFFE034660B9414693
:10144000204600F091F90028F1D0002383F31188A1
:10145000781B03B0BDE8F08FB9F1000F03D0019005
:101460002046C847019B8BF31188ED1A1E448AF36E
:101470001188DCE7026843681143016003B1184733
:10148000704700001430FFF743BF00004FF0FF33F8
:101490001430FFF73DBF00003830FFF7B9BF000040
:1014A0004FF0FF333830FFF7B3BF00001430FFF7C1
:1014B00009BF00004FF0FF311430FFF703BF0000F9
:1014C0003830FFF763BF00004FF0FF323830FFF7CE
:1014D0005DBF0000012914BF6FF0130000207047AA
:1014E000FFF740BD044B036000234360C0E90233B3
:1014F00001230374704700BFE027000810B53023B4
:10150000044683F31188FFF779FD0223002023743A
:1015100080F3118810BD000038B5C36904460D463C
:101520001BB904210844FFF7A5FF294604F1140064
:10153000FFF7ACFE002806DA201D4FF40061BDE87D
:101540003840FFF797BF38BD0023826803750369F1
:101550001B6899689142FBD25A6803604260106030
:101560005860704700238268037503691B68996897
:101570009142FBD85A68036042601060586070471F
:1015800008B50846302383F311880B7D032B05D063
:10159000042B0DD02BB983F3118808BD8B69002271
:1015A0001A604FF0FF338361FFF7CEFF0023F2E7AD
:1015B000D1E9003213605A60F3E70000FFF7C4BFBF
:1015C000054BD96808751868026853601A600122D3
:1015D000D8600275FEF716BF782C00200C4B30B592
:1015E000DD684B1C87B004460FD02B46094A68467D
:1015F00000F05CF92046FFF7E3FF009B13B168465B
:1016000000F05EF9A86907B030BDFFF7D9FFF9E730
:10161000782C002081150008044B1A68DB6890685C
:101620009B68984294BF002001207047782C0020CE
:10163000084B10B51C68D868226853601A600122F4
:10164000DC602275FFF78EFF01462046BDE81040A2
:10165000FEF7D8BE782C0020044B1A68DB6892682D
:101660009B689A4201D9FFF7E3BF7047782C0020AE
:1016700038B5074C012300250649074823706560EB
:1016800000F03AFC0223237085F3118838BD00BFB7
:10169000E02E00200C280008782C002000F046B92D
:1016A000EFF3118020B9EFF30583302282F3118824
:1016B0007047000010B530B9EFF30584C4F3080497
:1016C00014B180F3118810BDFFF7C6FF84F31188B1
:1016D000F9E700008B600223086108468B8270479F
:1016E0008368A3F1840243F8142C026943F8442C64
:1016F000426943F8402C094A43F8242CC268A3F1FC
:10170000200043F8182C022203F80C2C002203F8C6
:101710000B2C034A43F8102C704700BF1D0400082F
:10172000782C002008B5FFF7DBFFBDE80840FFF785
:1017300045BF0000024BDB6898610F20FFF740BFF8
:10174000782C0020302383F31188FFF7F3BF0000CB
:1017500008B50146302383F311880820FFF73EFFC8
:10176000002383F3118808BD064BDB6839B142685A
:1017700018605A60136043600420FFF72FBF4FF0DA
:10178000FF307047782C00200368984206D01A6812
:101790000260506018469961FFF710BF7047000063
:1017A000036810B59C68A2420CD85C688A600B6024
:1017B0004C602160596099688A1A9A604FF0FF3333
:1017C000836010BD121B1B68ECE700000A2938BFBC
:1017D0000A2170B504460D460A26601900F084FB04
:1017E00000F06CFB041BA54203D8751C04462E4672
:1017F000F3E70A2E04D90120BDE8704000F0BCBB1D
:1018000070BD0000F8B5144B0D460A2A4FF00A07C8
:10181000D96103F11001826038BF0A224160196961
:101820001446016048601861A81800F04DFB00F0F4
:1018300045FB431B0646A34206D37C1C28192746BA
:10184000354600F051FBF2E70A2F04D90120BDE82C
:10185000F84000F091BBF8BD782C0020F8B50646A2
:101860000D4600F02BFB0F4A134653F8107F9F42A2
:1018700006D12A4601463046BDE8F840FFF7C2BF10
:10188000D169BB68441A2C1928BF2C46A34202D93F
:101890002946FFF79BFF224631460348BDE8F84042
:1018A000FFF77EBF782C0020882C0020C0E903239E
:1018B000002310B45DF8044B4361FFF7CFBF000075
:1018C00010B5194C236998420DD08168D0E90032D7
:1018D00013605A609A680A449A60002303604FF0CC
:1018E000FF33A36110BD0268234643F8102F5360F5
:1018F0000022026022699A4203D1BDE8104000F044
:10190000EDBA936881680B44936000F0D7FA2269BE
:10191000E1699268441AA242E4D91144BDE810403A
:10192000091AFFF753BF00BF782C00202DE9F047BC
:10193000DFF8BC8008F110072C4ED8F8105000F0EA
:10194000BDFAD8F81C40AA68031B9A423ED814443A
:101950004FF00009D5E90032C8F81C4013605A6006
:10196000C5F80090D8F81030B34201D100F0B6FAB3
:1019700089F31188D5E9033128469847302383F34A
:1019800011886B69002BD8D000F098FA6A69A0EB37
:10199000040982464A450DD2022000F0EDFA0022E9
:1019A000D8F81030B34208D151462846BDE8F04778
:1019B000FFF728BF121A2244F2E712EB0909294661
:1019C000384638BF4A46FFF7EBFEB5E7D8F8103087
:1019D000B34208D01444C8F81C00211AA960BDE81D
:1019E000F047FFF7F3BEBDE8F08700BF882C00206A
:1019F000782C002000207047FEE7000070470000B0
:101A00004FF0FF3070470000BFF34F8F044B1A694F
:101A10005107FCD1D3F810215207F8D1704700BF0D
:101A20000020005208B50D4B1B78ABB9FFF7ECFF57
:101A30000B4BDA68D10704D50A4A5A6002F18832A2
:101A40005A60D3F80C21D20706D5064AC3F8042100
:101A500002F18832C3F8042108BD00BFE82E00203F
:101A6000002000522301674508B5114B1B78F3B9DC
:101A7000104B1A69510703D5DA6842F04002DA6068
:101A8000D3F81021520705D5D3F80C2142F04002BB
:101A9000C3F80C21FFF7B8FF064BDA6842F00102E9
:101AA000DA60D3F80C2142F00102C3F80C2108BD22
:101AB000E82E0020002000520F289ABF00F5806019
:101AC00040040020704700004FF4003070470000D1
:101AD000102070470F2808B50BD8FFF7EDFF00F571
:101AE00000330268013204D104308342F9D101206D
:101AF00008BD0020FCE700000F2870B5054645D85A
:101B0000FFF7CEFD224CFFF77FFF0646FFF78AFF67
:101B10004FF0FF33072D6361C4F8143120D82361DF
:101B2000FFF772FF2B0243F02403E360E36843F006
:101B30008003E36023695A07FCD42846FFF764FF5B
:101B40004FF40031FFF7B8FF00F002F93046FFF71D
:101B50008BFFFFF7AFFD2846BDE87040FFF7BABF27
:101B6000C4F81031FFF750FFA5F108031B0243F042
:101B70002403C4F80C31D4F80C3143F08003C4F8CA
:101B80000C31D4F810315B07FBD4D6E7002070BDD0
:101B9000002000522DE9F84F40EA020305460C46AA
:101BA0001746D80602D00020BDE8F88F27F01F079F
:101BB000DFF8D4B0FFF736FF2744BC4203D1012041
:101BC000FFF752FFF0E720222946204600F0CEFD25
:101BD00010B920352034F0E72B4605F120021E68AD
:101BE000711CE0D104339A42F9D1FFF759FD05F198
:101BF0007843234AB3F5801F224B28BF9A4603F14E
:101C0000040338BF9046A2F1080228BF9846A3F10A
:101C100008033ABF9146DA469946FFF7F5FEC8F841
:101C20000060A5EB040CD9F8002004F11C0142F07F
:101C30000202C9F80020221FDAF8006016F005063B
:101C4000FAD152F8043F8A424CF80230F4D1BFF383
:101C50004F8FFFF7D9FE4FF0FF32C8F80020D9F8B8
:101C6000002022F00202C9F80020FFF723FD202205
:101C70002146284600F07AFD0028AAD030469FE78A
:101C800014200052102100521020005210B5084CB0
:101C9000237828B11BB9FFF7C5FE0123237010BDBF
:101CA000002BFCD02070BDE81040FFF7DDBE00BF68
:101CB000E82E00200244074BD2B210B5904200D16A
:101CC00010BD441C00B253F8200041F8040BE0B2F0
:101CD000F4E700BF504000580E4B30B51C6F240491
:101CE00005D41C6F1C671C6F44F400441C670A4C2D
:101CF00002442368D2B243F480732360074B9042BE
:101D000000D130BD441C51F8045B00B243F82050B0
:101D1000E0B2F4E70044025800480258504000582E
:101D200007B5012201A90020FFF7C4FF019803B005
:101D30005DF804FB13B50446FFF7F2FFA04205D09F
:101D4000012201A900200194FFF7C6FF02B010BDD7
:101D50000144BFF34F8F064B884204D3BFF34F8F2C
:101D6000BFF36F8F7047C3F85C022030F4E700BF09
:101D700000ED00E0034B1A681AB9034AD2F8D024E8
:101D80001A607047EC2E00200040025808B5FFF79B
:101D9000F1FF024B1868C0F3806008BDEC2E0020F4
:101DA00070B5BFF34F8FBFF36F8F1A4A0021C2F88F
:101DB0005012BFF34F8FBFF36F8F536943F400335B
:101DC0005361BFF34F8FBFF36F8FC2F88410BFF31F
:101DD0004F8FD2F8803043F6E074C3F3C900C3F3E9
:101DE0004E335B0103EA0406014646EA8175013978
:101DF000C2F86052F9D2203B13F1200FF2D1BFF3A9
:101E00004F8F536943F480335361BFF34F8FBFF358
:101E10006F8F70BD00ED00E0FEE70000214B22480F
:101E2000224A70B5904237D3214BC11EDA1C121AD8
:101E300022F003028B4238BF00220021FEF7E6FFAA
:101E40001C4A0023C2F88430BFF34F8FD2F8803091
:101E500043F6E074C3F3C900C3F34E335B0103EAF6
:101E60000406014646EA81750139C2F86C52F9D27E
:101E7000203B13F1200FF2D1BFF34F8FBFF36F8FD1
:101E8000BFF34F8FBFF36F8F0023C2F85032BFF301
:101E90004F8FBFF36F8F70BD53F8041B40F8041BC6
:101EA000C0E700BF88290008702F0020702F002095
:101EB000702F002000ED00E000F07CB9014B586A63
:101EC000704700BF000C0040034B002258631A61AA
:101ED0000222DA60704700BF000C0040014B002274
:101EE000DA607047000C0040014B5863704700BF38
:101EF000000C0040FEE7000070B51B4B00250446B7
:101F000086B058600E468562016300F001F904F165
:101F10001003A560E562C4E904334FF0FF33C4E960
:101F20000044C4E90635FFF7C9FF2B46024604F119
:101F300034012046C4E9082380230C4A2565FFF7B5
:101F4000C9FB01230A4AE060009203756846726883
:101F50000192B268CDE90223064BCDE90435FFF7C3
:101F6000E1FB06B070BD00BFE02E0020182800087D
:101F70001D280008F51E0008024AD36A1843D062E3
:101F8000704700BF782C00204B6843608B688360EB
:101F9000CB68C3600B6943614B6903628B69436221
:101FA0000B6803607047000008B53A4B40F2FF71C0
:101FB0003948D3F888200A43C3F88820D3F888200A
:101FC00022F4FF6222F00702C3F88820D3F8883099
:101FD000324B1A6C0A431A649A6E0A439A66304A64
:101FE0009B6E1146FFF7D0FF00F5806002F11C01E7
:101FF000FFF7CAFF00F5806002F13801FFF7C4FF68
:1020000000F5806002F15401FFF7BEFF00F580602B
:1020100002F17001FFF7B8FF00F5806002F18C015A
:10202000FFF7B2FF00F5806002F1A801FFF7ACFFF7
:1020300000F5806002F1C401FFF7A6FF00F58060A3
:1020400002F1E001FFF7A0FF00F5806002F1FC0162
:10205000FFF79AFF02F58C7100F58060FFF794FF9F
:1020600000F066F90F4BD3F8902242F00102C3F85A
:102070009022D3F8942242F00102C3F89422052260
:10208000C3F898204FF06052C3F89C20064AC3F86A
:10209000A02008BD00440258000002580045025824
:1020A0002428000800ED00E01F00080308B500F038
:1020B00041FBFFF7DDFA0B4BDA6B42F04002DA63CB
:1020C0005A6E22F040025A665B6E074B1A6842F065
:1020D00008021A601A6842F004021A60BDE808405B
:1020E000FFF748BE0045025800180248704700003C
:1020F000EFF30983054968334A6B22F001024A6312
:1021000083F30988002383F31188704700EF00E010
:10211000302080F3118862B60D4B0E4AD96821F445
:10212000E0610904090C0A430B49DA60D3F8FC208A
:1021300042F08072C3F8FC20084AC2F8B01F116850
:1021400041F0010111602022DA7783F82200704704
:1021500000ED00E00003FA0555CEACC5001000E02C
:10216000302310B583F311880E4B5B6813F40063C2
:1021700014D0F1EE103AEFF309844FF08073683C0D
:10218000E361094BDB6B236684F30988FFF744FAAC
:1021900010B1064BA36110BD054BFBE783F311881B
:1021A000F9E700BF00ED00E000EF00E02F040008B9
:1021B000320400080E4B9A6C42F008029A641A6FBF
:1021C00042F008021A670B4A1B6FD36B43F00803F7
:1021D000D363C722084B9A624FF0FF32DA620022C3
:1021E0009A615A63DA605A6001225A611A60704734
:1021F000004502580010005C000C0040094A08B578
:102200001169D3680B40D9B29B076FEA01011161D4
:1022100007D5302383F31188FFF740FA002383F3B7
:10222000118808BD000C0040044BDA6B0243DA63EE
:102230005A6E104358665B6E704700BF00450258E7
:102240003A4B4FF0FF31D3F8802062F00042C3F8E0
:102250008020D3F8802002F00042C3F88020D3F819
:102260008020D3F88420C3F88410D3F8842000227F
:10227000C3F88420D3F88400D86F40F0FF4040F4C6
:10228000FF0040F4DF4040F07F00D867D86F20F0B7
:10229000FF4020F4FF0020F4DF4020F07F00D867EB
:1022A000D86FD3F888006FEA40506FEA5050C3F8F7
:1022B0008800D3F88800C0F30A00C3F88800D3F878
:1022C0008800D3F89000C3F89010D3F89000C3F8BA
:1022D0009020D3F89000D3F89400C3F89410D3F86A
:1022E0009400C3F89420D3F89400D3F89800C3F86E
:1022F0009810D3F89800C3F89820D3F89800D3F832
:102300008C00C3F88C10D3F88C00C3F88C20D3F861
:102310008C00D3F89C00C3F89C10D3F89C10C3F831
:102320009C20D3F89C3000F0BFB900BF0044025895
:1023300008B50122504BC3F80821504B5A6D42F0AA
:1023400002025A65DA6F42F00202DA670422DB6F9A
:102350004B4BDA605A689104FCD54A4A1A60012254
:102360009A60494ADA6000221A614FF440429A6149
:10237000434B9A699204FCD51A6842F480721A6041
:10238000424B1A6F12F4407F04D04FF480321A6728
:1023900000221A671A6842F001021A603B4B1A6861
:1023A0005007FCD500221A611A6912F03802FBD1DD
:1023B000012119604FF0804159605A67344ADA624E
:1023C000344A1A611A6842F480321A602F4B1A6834
:1023D0009103FCD51A6842F480521A601A6892047C
:1023E000FCD52D4A2D499A6200225A63196301F5E2
:1023F0007C01DA6301F5E77199635A64284A1A642B
:10240000284ADA621A6842F0A8521A601F4B1A680A
:1024100002F02852B2F1285FF9D148229A614FF4B4
:102420008862DA6140221A621F4ADA641F4A1A651A
:102430001F4A5A651F4A9A6532231F4A1360136860
:1024400003F00F03022BFAD1104A136943F0030380
:102450001361136903F03803182BFAD14FF00050C1
:10246000FFF7E2FE4FF08040FFF7DEFE4FF0004046
:10247000BDE80840FFF7D8BE008000510045025873
:102480000048025800C000F0040000010044025857
:102490000000FF01008890083220600063020901FB
:1024A000470E0508DD0BBF012000002000000110D1
:1024B0000910E00000010110002000524FF0B0426E
:1024C00008B5D2F8883003F00103C2F8883023B190
:1024D000044A13680BB150689847BDE80840FFF7FD
:1024E0003FBE00BFF02E00204FF0B04208B5D2F83A
:1024F000883003F00203C2F8883023B1044A93689D
:102500000BB1D0689847BDE80840FFF729BE00BF6F
:10251000F02E00204FF0B04208B5D2F8883003F01A
:102520000403C2F8883023B1044A13690BB150691F
:102530009847BDE80840FFF713BE00BFF02E00200B
:102540004FF0B04208B5D2F8883003F00803C2F863
:10255000883023B1044A93690BB1D0699847BDE82C
:102560000840FFF7FDBD00BFF02E00204FF0B04245
:1025700008B5D2F8883003F01003C2F8883023B1D0
:10258000044A136A0BB1506A9847BDE80840FFF748
:10259000E7BD00BFF02E00204FF0B04310B5D3F8D8
:1025A000884004F47872C3F88820A30604D5124A40
:1025B000936A0BB1D06A9847600604D50E4A136B34
:1025C0000BB1506B9847210604D50B4A936B0BB1A6
:1025D000D06B9847E20504D5074A136C0BB1506CD9
:1025E0009847A30504D5044A936C0BB1D06C984767
:1025F000BDE81040FFF7B4BDF02E00204FF0B0430F
:1026000010B5D3F8884004F47C42C3F888206205F2
:1026100004D5164A136D0BB1506D9847230504D5A8
:10262000124A936D0BB1D06D9847E00404D50F4A60
:10263000136E0BB1506E9847A10404D50B4A936EEC
:102640000BB1D06E9847620404D5084A136F0BB1E2
:10265000506F9847230404D5044A936F0BB1D06F91
:102660009847BDE81040FFF77BBD00BFF02E00206B
:1026700008B50348FEF71CFDBDE80840FFF770BD34
:10268000A023002008B50348FEF712FDBDE808406E
:10269000FFF766BD0C24002008B5FFF7AFFDBDE8CD
:1026A0000840FFF75DBD0000062108B5084600F0B0
:1026B0002BF80621072000F027F80621082000F05B
:1026C00023F80621092000F01FF806210A2000F057
:1026D0001BF80621172000F017F80621282000F02B
:1026E00013F809217A2000F00FF80721322000F0BA
:1026F0000BF80C21522000F007F80C215320BDE804
:10270000084000F001B80000090100F16043012217
:1027100003F56143C9B283F8001300F01F039A4028
:1027200043099B0003F1604303F56143C3F8802133
:102730001A60704708B5FFF783FD00F009F8FEF74F
:10274000CFFEFFF7D3FCBDE80840FFF7B5BB0000A4
:102750000023054A19460133102BC2E9001102F18A
:102760000802F8D1704700BFF02E002010B50139E3
:102770000244904201D1002005E0037811F8014F96
:10278000A34201D0181B10BD0130F2E753544D3362
:102790003248373F3F3F0053544D33324837337848
:1027A0002F3732780053544D3332483734332F3774
:1027B00035332F373530000001105A00031059000F
:1027C0000120580003205600009600000000000081
:1027D00000000000000000000000000000000000F9
:1027E00000000000A11400088D140008C91400089E
:1027F000B5140008C1140008AD14000899140008AD
:1028000085140008D514000863300000082800086B
:10281000D02C0020E02E00206D61696E0069646C90
:10282000650000000000002800000000AAAAAAAA73
:1028300000000024FFFF0000000000000000000076
:102840000000000000000000AAAAAAAA00000000E0
:10285000FFFF00000000000000000000000000007A
:1028600000000000AAAAAAAA00000000FFFF0000C2
:102870000000000000000000000010000000000048
:10288000AAAAAAAA00000000FFFF000000000000A2
:10289000000000000A80020000000000AAAAAAAA04
:1028A00005400100FFFF00008800007007000000E5
:1028B0000000000000000000AAAAAAAA0000000070
:1028C000FFFF00000000000000000000000000000A
:1028D00000000000AAAAAAAA00000000FFFF000052
:1028E00000000000000000000000000000000000E8
:1028F000AAAAAAAA00000000FFFF00000000000032
:10290000000000000000000000000000AAAAAAAA1F
:1029100000000000FFFF00000000000000000000B9
:102920000000000000000000AAAAAAAA00000000FF
:10293000FFFF000000000000000000000000000099
:1029400000000000AAAAAAAA00000000FFFF0000E1
:1029500000000000000000002E0400000000000045
:1029600000001A0000000000FF000000A02300206B
:10297000000000008C27000883040000972700084F
:0829800050040000A527000827
:00000001FF
